S11BB8007EB8CD7EB8667EB8927EBAA87EBA7C7EBA790442BB390444FE
S11BB818BC660447BB64044CBD49044DB9FB054D56BF2F044FBA530433
S11BB83050BD1B0452BABF054849B8C0054859B8C80454BB870456BD20
S11BB8485A074348434BBE120750524F47BE800756455246BF4707587E
S11BB86054414CBF73FE378D1224FC847F27F8817F27F4D6FF26028DFE
S11BB878193339961148250348240396120D3937D611C52027FA9713ED
S11BB8903339378DF2D6FF2602D6E6810D2708811027EDC40320025422
S11BB8A8545A2BE4364F8DD73220F6CEBFA3BDBAA8CE411B0926FD39B8
S11BB8C0CC4F0697E6D71039CC000520F68E00C69FF5CE00F76F0008A3
S11BB8D88C010026F8CC10078DE1860A97118DCBCEBFADBDBAAF86D012
S11BB8F097F4CEEFEADFDB7C00088E00DA7F00FFBDBAB3862BBDB89204
S11BB908BDB9A925ED270ABDB99C25E6CEB9FF206CCEBB82812E27654C
S11BB920CEBA48812F275E9FE27F00E18D5D27137C00E136308C009022
S11BB9382F23BDB9A92524261C20E997E7CEB812DFE4DEE43CE6003AF7
S11BB950DFE4C003D1E1270D38C1FB26EDCEBFABBDBAAF2095DEE2DFB6
S11BB968EA3808A6003CDEEAA10027033820D309DFEA5A26EC38089EDD
S11BB980E2EE0096E7AD0025D420D8812C270A81202706810D270281DC
S11BB9982D398D11230AC1042F397D00ED27340D39C6F020015FCE0026
S11BB9B000DFEADFECCE00EA8D252517C6046801690024037C00ED5ABB
S11BB9C826F4AA01A7017C00EC20E5811826020D39DEEAD6EC0C39BDF6
S11BB9E0B86681302BF181392F0D5D2BEA81412BE681462EE280078443
S11BB9F80F5F398D9D2F52DEEA812F2704812026488D77DFE83C5F8D3C
S11BBA109C38253E2707D6EBBDBA982535810D2731812C26030820E3C4
S11BBA28812026030820DA810A260608BDBAB7200D815E2603092004E7
S11BBA40812F260D8D6DDFE8CE00E88D2CDEE820B80D39BDBD0325F958
S11BBA58DCEA83000193E8C17F22054D270620E981FF26E5D7EC8D4305
S11BBA70CE00EC8D078D3C20CF8D07088D048620203AA600368D0332E9
S11BBA88200444444444840F8B90198940192024E700E10027B4CEBF51
S11BBAA0B88D0C20AC8D1508A600810426F7398D0220F5860A8D0586F6
S11BBAB80D8D014F7EB8928D668DF0CE00EE5F3CCEBFD23AA6008D62CB
S11BBAD0A601387D00E1270B4D27038DA5088D9C082004378D0833CB1B
S11BBAE802C10C26DA39363CBDB9AD3833251B271DBDB98B26145D27F7
S11BBB000936DCEAED0032082004D6EBE700810D261338334F398120D6
S11BBB1826F85D2605BDBA7C2003BDBA7908398D8A7C00E18D957F000F
S11BBB30E1398D02862D7EB892810D270F812D2716BDB99A230F810D56
S11BBB48260BDFF7BDBAB3CE00F77EBA790D39BDB866810D26F74F5FC0
S11BBB60DDF720E8810D270EBDB99A23E8810D26E47F00FDDFEEBDBAB7
S11BBB78B396FD2603BDBC2A2015CE00012009810D27F7BDB9AD2FC5AF
S11BBB90DFFB27C17C00FD2048C618DE093ADF0B397C00088DF3308E12
S11BBBA800DA8D56BDBC1ADEFB26097F00FD8D72251D202509DFFB261E
S11BBBC0037F00FDCE0000BDBCEE27F1CEBFCEBDBAAFDEEABDBA7CBDA4
S11BBBD8BB2996FD26037EB8FA9EF5DEEE3CDEF03CDCF2363796F436E1
S11BBBF096FD270DDEEEDFEA860297017A00088D983BA60097F4EC01BD
S11BBC0897F3D7F2EC03DDF0EC05DDEEC6063ADFF53996FA270B96F9F1
S11BBC20DEF72702A7007F00FA3996FA265CDEF7270DA600C63FBDBA74
S11BBC3898250497F997FA39308E00DA8DBCDEEE09DFEEDFEA96FA27D2
S11BBC50098DC79CEA26034C20044F5FDDFB97FDBDBB277EB8FADEE8AD
S11BBC683C810D270A8D7C2316DFE8810D2615DCE8C4F0830010DDE823
S11BBC80C30020DDEA201938DFE80D398D5D23F7DCE8C4F0D7E993EAC7
S11BBC9822ED96EB84F097EBBDBAB38D49260538DFE84F39BDBAB3CE60
S11BBCB000E8BDBA79DEE8C610BDBA7C085A26F9BDBA7EC610DEE8A659
S11BBCC800847F81202D0481612D02862EBDB892085A26EBDCEA93E80B
S11BBCE027C5DFE87D00E926BA20B57EB99A36BDB87B847F81172607BB
S11BBCF8BDB87B24FB847F81183239810D27128DE2230EDFE8810D2737
S11BBD10088DD82304810D27010D397F00E78DE325F8BDBAB38610973D
S11BBD28FF4CD6E726014CBDB892BDBD5E4636CEBFA8BDB8B6BDBCEE62
S11BBD40BDBCEE7F00FF324939C601D7E7CE0000DFEA810D27CC8DB96B
S11BBD5820C8C6FF20ED5D2758DCEADDE8BDB866815326F9BDB8668184
S11BBD70392731813126F17F00E18D29C002D7EC8D23378D2032D3E841
S11BBD883736388D187A00EC270E7D00E72B02E700E10026060820EB22
S11BBDA04C27C20D395FBDB9DFC6103D375FBDB9DF331B169BE197E102
S11BBDB839C6194FBDB8925A26F9DCEAD0E992E82604C1182502C61788
S11BBDD0CB04D7E7C003D7ECCEBFBFBDBAAF5FCE00E78D29CE00E88DC5
S11BBDE824088D21DEE88D1D087A00EC26F8DFE85337308D1033DEE852
S11BBE00099CEA26BDCEBFC2BDBAAF4F39EB007EBA82810D2773BDBD70
S11BBE18039CE8256CCCFF869714D7ECDEE80908E60027054F8D0F273C
S11BBE30089CEA26F27F00FE397F00FE0D3936373CD6EC2A08CEBFEAC3
S11BBE48BDBAAFC40F2605C606BDBAB330BDBA7908BDBA82862FBDB879
S11BBE609208BDBA7CBDBA7E5A38D7EC3332BDBCEE39CEBFE43CBDBAC6
S11BBE78AFBDB86638815939810D2705BDBF0624020D39BDBE1DD6ECD7
S11BBE902B07CEBFDE8DDE26F08DD726EC86FE9714DEE83CDEDD093CD1
S11BBEA8389CDF26137D00FE2B8338DFE88DBB27FC814E26F87EBF4F86
S11BBEC008A6003CDEE87D00FE2B1AA70086FC97149608DCDBD309DD14
S11BBED80B9608844027FA86FE9714200DE600112708BDBE3E26033824
S11BBEF020BB08DFE820B1BDB99A2F8DDFDD810D2787BDBD03398DEFC5
S11BBF08250EDCE8DDDF81F82406DFE893DD24037EBE89D3E825F9DDEE
S11BBF20EADCDD81F824F196E881F825EB0C398DC625E5DEDD0908A6B9
S11BBF38003CDEEAA70008DFEA389CE826F039810D27528DB9254ECCDA
S11BBF50FF869714D7ECD7FE7EBEA4302920322E3435202031292034FD
S11BBF682E39310D0A5854414C3D04CEBF5BBDBAAF8630D6DBC17727C0
S11BBF80014CBDB892BDBA7EBDB866810D2712CE77EA80302709CEEFEE
S11BBF98EA810127020D39DFDB0C39103A1039041413043F0450524FBD
S11BBFB042554720312E30044E4F20434847045331045339303330307A
S11BBFC8303046430D044F502D04500158014100420043005301434844
S11BBFE0473F20045057523F2004414452204550522F56414C0D0A0434
S10BBFF8009ABC40BBA1B80093
S9030000FC
